:020000040000FA
:04000000EB303A287F
:040004000034003490
:08000800A000030EA100831209
:1000100005191128831601178312B2308100B1012E
:100020002C2883160113831203140B190310A80D37
:10003000A90DAA0DAB0DAC0DAC16FF302C02031DA3
:100040002C28FA302B02031D2C2832152A08AF0069
:100050002908AE002808AD008B100B11210E83007B
:06006000A00E200E0900B5
:0C007400203084008001840A80300402E7
:10008000031C3C28152283160C308505870183123A
:10009000850187010730990000309A0010308316DF
:1000A0008E008312603083168F0083120030831617
:1000B000910000008312C830831681008312313012
:1000C0009000003083168C00831210308B00982330
:1000D00081018E018F010B118B100B108C018B177E
:1000E0007F2032198B20B40B7D280310851903144F
:1000F000BA0DF0303A0203195E21FF237028640024
:100100003310B10A311F8A28AC01AB01AA01A90141
:10011000A801B101080032110130B7008B13203063
:100120003707371A313E83169B001C141A088312B6
:10013000A40010303707371A313E83169B001C1479
:100140001A088312A300A6000230A6060030370763
:10015000371A313E83169B001C141A088312A20022
:10016000A7000130A7068B17331CBC2822090339CE
:10017000A200A309A409A50924082F02031D5829D8
:1001800023082E02031D582922082D02031D582979
:1001900001303702031DD1283E18D1283E143F14E8
:1001A000302202303702031DDA28BE18DA28BE14C6
:1001B0003F14422203303702031DE3283E19E3288F
:1001C0003E153F14542204303702031DEC28BE199B
:1001D000EC28BE153F14662205303702031DF528B2
:1001E0003E1AF5283E163F14782206303702031DCA
:1001F000FE28BE1AFE28BE163F1489220730370299
:10020000031D07293E1B07293E173F149A22083079
:100210003702031D1029BE1B1029BE173F14AB2245
:1002200009303702031D19295E1819295E143F147D
:10023000BC220A303702031D2229DE182229DE14CF
:100240003F14CD220B303702031D2B295E192B29B9
:100250005E153F14DE220C303702031D3429DE19EF
:100260003429DE153F14EF220D303702031D3D29DE
:100270005E1A3D295E163F1400230E303702031D1F
:100280004629DE1A4629DE163F1411230F303702A5
:10029000031D4F295E1B4F295E173F142223103088
:1002A0003702031D5829DE1B5829DE173F1433235C
:1002B000B70A11303702031808008E280130B60043
:1002C000B400B500B70085018701B21395237F20E4
:1002D000B40B7729031085190314BA0DF0303A02D4
:1002E0000319A529B50B77299630B500B121321D28
:1002F00067293211331C81292D090339AD00AE095C
:10030000AF092F1C67292D083002031967292D0812
:10031000B0002E1E67298B1320303707371A313E65
:10032000BC002F08BB00002210303707371A313EBF
:10033000BC002E08BB00002200303707371A313EC0
:10034000BC002D08BB0000228B1785018701B70A6E
:10035000B6010130B50011303702031C672998231C
:100360000800013037020319452302303702031910
:100370004A230330370203194F230430370203198D
:100380005423053037020319592306303702031965
:100390005E2307303702031963230830370203193D
:1003A00068230930370203196D230A303702031915
:1003B00072230B303702031977230C3037020319ED
:1003C0007C230D303702031981230E3037020319C5
:1003D00086230F30370203198B231030370203199D
:1003E000902308003F1C08003F101030BC003E085E
:1003F000BB0000223030BC005E08BB0000220800B9
:100400008B133B0883161C159A0083123C08831635
:100410009B0055309D00AA309D009C1464009C18E0
:100420000E2A1C1183128B170800831610309B00B4
:100430001C141A088312BE00831630309B001C1453
:100440001A088312DE00FF30C800CA15CB15CC1580
:10045000CD15CE15CF15D015D115D215D315080051
:100460000130BE050030DE052030C405C00000307C
:10047000C200C6000030C505C1000030C300C7007F
:100480005F1008000230BE050030DE052030C405D4
:10049000C0002030C200C6000030C505C1000030D9
:1004A000C300C7005F1008000430BE050030DE0541
:1004B0005030C405C0000030C200C6000030C50581
:1004C000C1000030C300C7005F1008000830BE053F
:1004D0000030DE055030C405C0001030C200C60038
:1004E0000030C505C1000030C300C7005F10080020
:1004F0001030BE050030DE050330C405C0000030FA
:10050000C200C6008030C505C1000030C300C7006E
:1005100008002030BE050030DE050630C405C000EE
:100520000030C200C6008030C505C1000030C300E5
:10053000C70008004030BE050030DE050A30C405A3
:10054000C0000030C200C6008030C505C1000030C8
:10055000C300C70008008030BE050030DE0509304A
:10056000C405C0000030C200C6008030C505C1000F
:100570000030C300C70008000030BE050130DE05B2
:100580009030C405C0000030C200C6000030C50570
:10059000C1000030C300C70008000030BE050230B3
:1005A000DE059030C405C0001030C200C600003027
:1005B000C505C1000030C300C70008000030BE05FB
:1005C0000430DE051030C405C0000030C200C60093
:1005D0004030C505C1000030C300C700080000302E
:1005E000BE050830DE051030C405C0001030C20062
:1005F000C6004030C505C1000030C300C700080078
:100600000030BE051030DE051330C405C0000030D8
:10061000C200C6000030C505C1000030C300C700DD
:1006200008000030BE052030DE052330C405C000C0
:100630000030C200C6000030C505C1000030C30054
:10064000C70008000030BE054030DE051330C40589
:10065000C0001030C200C6000030C505C100003027
:10066000C300C70008000030BE058030DE0523301F
:10067000C405C0002030C200C6000030C505C1005E
:100680000030C300C70008000800003085060430B1
:100690008706080000308506043087060800003011
:1006A000850603308706080000308506033087067C
:1006B000080030308506083087060800213085069E
:1006C00008308706080022308506083087060800B3
:1006D0001230850608308706080000308506223073
:1006E00087060800003085062230870608000030A3
:1006F000850612308706080000308506123087060E
:100700000800303085060230870608003030850644
:10071000043087060800303085060230870608005E
:10072000303085060430870608003E18452308004F
:100730003E183022BE1842223E195422BE196622AB
:100740003E1A7822BE1A89223E1B9A22BE1BAB2279
:100750005E18BC22DE18CD225E19DE22DE19EF22E1
:100760005E1A0023DE1A11235E1B2223DE1B3323B5
:100770000800B601B401B5013D1CC12BBD01BD147B
:10078000C32BBD013D143D08B6006400C72BC82B28
:10079000C92BCA2BCB2BFF30B51B8500B51F85019C
:1007A000B40BC52BB50BC52B0310B60CB608031D37
:1007B000C52B0030BC003D08BB000022080005121C
:1007C0005C180516DC1C8512DC1885165C1D0510EE
:1007D0005C190514DC1D8510DC1985145C1E87105E
:1007E0005C1A8714DC1E0711DC1A07155C1F071042
:1007F0005C1B0714DC1F8712DC1B871608008F08A0
:10080000031908008F0178308E00C80F3D2EC80AEA
:10081000DF19312C441C312C461C222CCA1C132CF1
:10082000CA014A153F2C4A1D182CCA01CA153F2C73
:10083000CA1D1D2CCA014A163F2C4A1E3F2CCA0154
:10084000CA143F2C4A1D272CCA014A163F2CCA1D28
:100850002C2CCA014A163F2C4A1E3F2CCA01CA142E
:100860003F2CCA1C362CCA014A153F2C4A1D3B2C72
:10087000CA01CA153F2C4A1E3F2CCA014A15DF196E
:10088000682CC41C682CC61C592CCB1C4A2CCB01D0
:100890004B15762C4B1D4F2CCB01CB15762CCB1D3D
:1008A000542CCB014B16762C4B1E762CCB01CB1443
:1008B000762C4B1D5E2CCB014B16762CCB1D632C5E
:1008C000CB014B16762C4B1E762CCB01CB14762C01
:1008D000CB1C6D2CCB014B15762C4B1D722CCB01F8
:1008E000CB15762C4B1E762CCB014B15DF199F2C8C
:1008F000441D9F2C461D902CCC1C812CCC014C15EA
:10090000AD2C4C1D862CCC01CC15AD2CCC1D8B2CCC
:10091000CC014C16AD2C4C1EAD2CCC01CC14AD2C06
:100920004C1D952CCC014C16AD2CCC1D9A2CCC0119
:100930004C16AD2C4C1EAD2CCC01CC14AD2CCC1CCB
:10094000A42CCC014C15AD2C4C1DA92CCC01CC15E4
:10095000AD2C4C1EAD2CCC014C15DF19D72CC41D71
:10096000D72CC61DC82CCD1CB92CCD014D155F133D
:10097000E52C4D1DBE2CCD01CD15E52CCD1DC32C78
:10098000CD014D16E52C4D1EE52CCD01CD14E52CE9
:100990004D1DCD2CCD014D16E52CCD1DD22CCD01FC
:1009A0004D16E52C4D1EE52CCD01CD14E52CCD1CAE
:1009B000DC2CCD014D15E52C4D1DE12CCD01CD15C7
:1009C000E52C4D1EE52CCD014D15DF19102D5F1BBB
:1009D000102D441E102D461E012DCE1CF22CCE01D2
:1009E0004E151E2D4E1DF72CCE01CE151E2DCE1DE3
:1009F000FC2CCE014E161E2D4E1E1E2DCE01CE14E9
:100A00001E2D4E1D062DCE014E161E2DCE1D0B2D5C
:100A1000CE014E161E2D4E1E1E2DCE01CE141E2DA5
:100A2000CE1C152DCE014E151E2D4E1D1A2DCE019C
:100A3000CE151E2D4E1E1E2DCE014E15DF19472D33
:100A4000C41E472DC61E382DCF1C292DCF014F1592
:100A5000552D4F1D2E2DCF01CF15552DCF1D332DCB
:100A6000CF014F16552D4F1E552DCF01CF14552DAB
:100A70004F1D3D2DCF014F16552DCF1D422DCF01BE
:100A80004F16552D4F1E552DCF01CF14552DCF1C70
:100A90004C2DCF014F15552D4F1D512DCF01CF1589
:100AA000552D4F1E552DCF014F15DF197E2D441F9B
:100AB0007E2D461F6F2DD01C602DD00150158C2D22
:100AC000501D652DD001D0158C2DD01D6A2DD00163
:100AD00050168C2D501E8C2DD001D0148C2D501DF5
:100AE000742DD00150168C2DD01D792DD0015016AB
:100AF0008C2D501E8C2DD001D0148C2DD01C832D0C
:100B0000D00150158C2D501D882DD001D0158C2D65
:100B1000501E8C2DD0015015DF19B52DC41FB52DD9
:100B2000C61FA62DD11C972DD1015115C32D511DC6
:100B30009C2DD101D115C32DD11DA12DD10151164F
:100B4000C32D511EC32DD101D114C32D511DAB2D69
:100B5000D1015116C32DD11DB02DD1015116C32D78
:100B6000511EC32DD101D114C32DD11CBA2DD101D9
:100B70005115C32D511DBF2DD101D115C32D511EAE
:100B8000C32DD1015115DF19ED2D451FED2D471F47
:100B9000DE2DD21CCF2DD2015215DF13FB2D521D9D
:100BA000D42DD201D215FB2DD21DD92DD201521632
:100BB000FB2D521EFB2DD201D214FB2D521DE32D15
:100BC000D2015216FB2DD21DE82DD2015216FB2D5B
:100BD000521EFB2DD201D214FB2DD21CF22DD201BC
:100BE0005215FB2D521DF72DD201D215FB2D521E91
:100BF000FB2DD2015215DF19262EDF1B262EC51F15
:100C0000262EC71F172ED31C082ED3015315342EA2
:100C1000531D0D2ED301D315342ED31D122ED30107
:100C20005316342E531E342ED301D314342E531D99
:100C30001C2ED3015316342ED31D212ED30153164F
:100C4000342E531E342ED301D314342ED31C2B2E0A
:100C5000D3015315342E531D302ED301D315342E0A
:100C6000531E342ED3015315F2214008C40041080D
:100C7000C5005F18DF145F1CDF104808C9000C3086
:100C80004A05031D05120C304B05031D85120C305F
:100C90004C05031D05100C304D05031D85100C304F
:100CA0004E05031D87100C304F05031D07110C3036
:100CB0005005031D07100C305105031D87120C3021
:100CC0005205031D07120C305305031D87114908F7
:100CD0000E020318972E12304A05031D0516123016
:100CE0004B05031D851612304C05031D05141230EB
:100CF0004D05031D851412304E05031D8714123057
:100D00004F05031D071512305005031D071412303F
:100D10005105031D871612305205031D07161230A8
:100D20005305031D8715FF304802031908008F087B
:100D3000031D08007F2049080E02031C972E18305F
:100D40004A05031D051206304A05031D0516183015
:100D50004B05031D851206304B05031D8516183003
:100D60004C05031D051006304C05031D05141830F5
:100D70004D05031D851006304D05031D85141830E3
:100D80004E05031D871006304E05031D87141830CD
:100D90004F05031D071106304F05031D07151830B9
:100DA0005005031D071006305005031D07141830A9
:100DB0005105031D871206305105031D8716183093
:100DC0005205031D071206305205031D0716183081
:100DD0005305031D871106305305031D87150800B1
:084000000B00030007000100A2
:02400E00CC33B1
:10420000010078007A007C007E007B0079007F004E
:104210007D007A0078007E007C007D007F007900C0
:104220000100F200F600FA00FE00F200F600FA00CB
:10423000FE00F200F600FA00FE00F200F600FA00BE
:10424000FF00050005000500050009000900090040
:1042500009000D000D000D000D00110011001100EE
:104260000000FF00FF00FF00FF00FF00FF00FF0055
:10427000FF00FF00FF00FF00FF00FF00FF00FF0046
:10428000FF007B00FF00FF00FF00FF00FF00FF00BA
:10429000FF00FF00FF00FF00FF00FF00FF00FF0026
:1042A000FF00FE00FF00FF00FF00FF00FF00FF0017
:1042B000FF00FF00FF00FF00FF00FF00FF00FF0006
:1042C000FF001100FF00FF00FF00FF00FF00FF00E4
:1042D000FF00FF00FF00FF00FF00FF00FF00FF00E6
:1042E000FF00FF00FF00FF00FF00FF00FF00FF00D6
:1042F000FF00FF00FF00FF00FF00FF00FF00DD00E8
:00000001FF
